:020000040800F2
:10000000D01B0020A9010008E1100008C108000869
:1000100000000000000000000000000000000000E0
:10002000000000000000000000000000591400085B
:100030000000000000000000E3100008591500084F
:10004000BB010008BB010008BB010008BB010008A0
:10005000BB010008BB010008BB010008BB01000890
:1000600000000000BB010008BB010008BB01000844
:10007000BB010008BB010008BB0100080000000034
:10008000BB010008BB010008000000005D1600086D
:1000900091160008F91600081D170008BB0100089A
:1000A000BB010008BB010008BB0100087D17000868
:1000B0000D18000800000000000000000000000013
:1000C000BB01000800000000BB01000800F002F8BE
:1000D00000F03EF80CA030C8083824182D18671E10
:1000E000A246AB4654465D46AC4201D100F030F822
:1000F0007E460F3EB6460FCC0126334200D0FB1A97
:100100003343A246AB461847183D0000383D000077
:10011000103A02D378C878C1FAD8520701D330C850
:1001200030C101D504680C60704700000023002432
:1001300000250026103A01D378C1FBD8520700D31E
:1001400030C100D50B6070471FB51FBD10B510BD85
:1001500000F0A1F91146FFF7F7FF02F0ADFA00F049
:10016000B9F903B4FFF7F2FF03BC00F0BFF90000D8
:1001700070B505460C46164602E00FCC0FC5103E82
:10018000102EFAD2082E02D303CC03C5083E042E4B
:1001900007D301CC01C5361F03E021782970641C08
:1001A0006D1C761EF9D270BD07488047074800478E
:1001B000FEE7FEE7FEE7FEE7FEE7FEE70448054947
:1001C000054A064B704700006D150008CD00000879
:1001D000D0130020D01B0020D0170020D017002003
:1001E000F8B5042A2CD3830712D00B78491C03706E
:1001F000401C521E83070BD00B78491C0370401C17
:10020000521E830704D00B78491C0370401C521EF9
:100210008B079B0F05D0C91ADF002023DE1B08C9FE
:100220000AE0FFF7A5FFF8BD1D4608C9FD401C46C2
:10023000B4402C4310C0121F042AF5D2F308C91A87
:10024000521EF0D40B78491C0370401C521EEAD495
:100250000B78491C0370401C012AE4D40978017012
:10026000F8BD01E004C0091F0429FBD28B0701D5AA
:100270000280801CC90700D00270704700290BD093
:10028000C30702D00270401C491E022904D3830711
:1002900002D50280801C891EE3E70022EEE70022DF
:1002A000DFE7704770477047F0B5FF252D04C6099A
:1002B000C209FF2704462E400137CB093E43484080
:1002C0002A402B400746002A6BD0002B69D0AA4257
:1002D00067D0AB4265D0002800DA32460125ED0533
:1002E00029432C4309022002090AD21A4B0C7F240D
:1002F000E31A434C000A7C44E35C7D242404121975
:1003000014145B00A218884201D3521C00E0400084
:1003100049420C465C4324115C43DB016415E3183D
:10032000040A5C43C502200D0C4644436419250AA7
:100330005D432303EC0C0D46654300030019EB18E5
:100340004C42A34201D35B18401CD4052018002B5B
:1003500007D05B00C91804D3401C002901D1400814
:1003600040003F2189048A4209D3002A08DC110693
:10037000090F04D0032149074018C00FC007F0BD82
:1003800001224100120689187F2252069142F6D2BC
:1003900005214907C84201D59010F0BDFF20C005D6
:1003A000F0BD002F00DA32461648AA4207D2AB420F
:1003B00005D21902090E17D0F80FC007F0BDFF25AE
:1003C00063002D06AB42F9D84900A942F6D8AB42EA
:1003D00001D1A942F2D0A94201D1002101E061007E
:1003E0004908D0050843F0BD1102090EFBD0FF20DB
:1003F0000243D005F0BD0A460146104654E700000E
:10040000FE3700000000C07F0102C21504D00123A6
:10041000DB071943002A0ADB9E239A1A02D40846F6
:10042000D0407047FF2241001206914201D90020BE
:100430007047C017C04370471F22030C02D10F2220
:1004400000041CD0030E01D10002083A030F01D1B1
:100450000001121F830F01D18000921E002801DBD2
:100460004000521ED2055118021251181922904014
:1004700004D3491C002801D14908490008467047A7
:10048000C10FC90700D04042012292071143D3E7B0
:1004900001218907D0E7754600F024F8AE46050033
:1004A00069465346C008C000854618B020B5FFF71E
:1004B00085FE60BCB64600260027C0C5C0C5C0C5C5
:1004C000C0C5C0C5C0C5C0C5C0C5403D490849007C
:1004D0008D46704710B50446C046C0462046FFF71B
:1004E00040FE10BD004870479000002001491820D0
:1004F000ABBEFEE72600020070470000B0B588B032
:10050000974802F073FD40F2005002F06FFD0024A6
:10051000204601F0D9FA01AD40F200102883AC76F4
:100520000E4901910E49891C039140F2004104914A
:10053000029042F20000069008200590204601F04B
:10054000BBFA2046294601F0E9FA204601F01EFBDD
:10055000204601F0A9FA08B0B0BDC0464C240140C5
:100560003C01002070B514460D460646200407D015
:10057000B0B200F007F82870641E6D1C761CF5E719
:1005800070BD000070B5044600F054F9A020214D64
:10059000A847214EB047200AA847B047E0B2A84775
:1005A000B04700F047F9A120A847B047002000F06D
:1005B00089F9044600F05EF9204670BD70B5144616
:1005C0000D460646200407D02978B0B200F006F8A0
:1005D000641E6D1C761CF5E770BD0000F8B50C4676
:1005E000054600F027F9A0200A4EB0470A4FB84749
:1005F000280AB047B847E8B2B047B8472046B047E6
:10060000B84700F037F90A20F8BC02BC8E4600F06B
:10061000B9B8C046290900088D090008F0B50B4D8E
:1006200000210B4A0B4B0C4684420DD0165D7540E1
:100630000E46072E06D86F08ED0700D05F403D46F6
:10064000761CF6E7641CEFE7A8B2F0BDFFFF0000E0
:10065000B50A002001A00000984800218170704771
:10066000F0B587B040F2005011303C4CA04740F24A
:1006700000501230A0473A48A04740F20050A0472F
:100680000620059002F0BCFB09200690C00603245A
:1006900004940025F32321462A4601F0CDFF31487A
:1006A00021462A46234601F0C7FF01F037F9FFF73C
:1006B00025FF012640F20010314601F0C5F9022065
:1006C0000190314601F0C0F9072003904104304603
:1006D00001F044F9284601F015F9284601F098F98F
:1006E00008210291304601F0EDF805241E4F2846FE
:1006F00029462246B847304631462246B8470425A7
:10070000019829462246B847049821462246B84710
:100710002846059D29462246B8472046039F39466C
:100720002246114B98472846029922460E4DA8476B
:10073000384606992246A84701F006F901F004F967
:1007400001F0B0F801F0F8F8304601F06BF93046EE
:1007500007B0F0BC02BC8E4601F064B9ED2F000872
:1007600009060000000400488519000838B1044952
:1007700041430F204003B1FBF0F10A20484370478A
:10078000E880000081B00090034800990160016892
:100790000029FCD101B07047F80A002081B0009018
:1007A000009801B07047F8B505460920C4062046F8
:1007B00040F6000101F035FF204641F2000101F052
:1007C00030FF00270126082F20D02846F840C00718
:1007D00005D0204648F2000101F025FF04E0204644
:1007E00048F2000101F01DFF3046FFF7D7FF204619
:1007F00040F6000101F017FF3046FFF7CFFF20461B
:1008000040F6000101F00DFF7F1CDCE701252846C2
:10081000FFF7C4FF204641F2000101F004FF284623
:10082000FFF7BCFF204641F20001F8BC04BC96462D
:1008300001F0F7BEF8B500F05BFE814C01262046C2
:10084000314601F0F0FE02252046294601F0EBFE7C
:1008500004273846FFF7A2FF2046314601F0E1FEAB
:100860003846FFF79BFF20462946F8BC04BC964655
:1008700001F0D7BEF8B500F03BFE714C02252046D2
:10088000294601F0CEFE01262046314601F0C9FE80
:1008900004273846FFF782FF2046294601F0C3FEB1
:1008A0002046314601F0BFFE3846F8BC02BC8E46F9
:1008B000FFF774BF014880787047C046F000002001
:1008C000FEE70000FEB5009000F00CFE00210226BD
:1008D000012001900C46019D07291CD8584F38462D
:1008E0000291314601F09DFE3046FFF757FF384632
:1008F000314601F098FE3846294601F098FE274619
:1009000004462846FFF74AFF0299601E844178009A
:100910000419491CE0E7009810B100F0A5FD01E0C2
:1009200000F0C2FDE0B2FEBDFEB5044600F0E0FD01
:1009300043480226314601F074FE00270120019051
:10094000072F1FD860B2002802943D4D284603D4DB
:10095000019901F066FE02E0019901F064FE304663
:10096000094CA0472846314601F05DFE3046A047BD
:100970002846314601F055FE3046A0477F1C029CB8
:100980006400DDE7FEBDC0469D07000870B500F0BD
:10099000A9FD2B4C0221204601F045FE01252846E9
:1009A000FFF7FCFE00262046294601F040FE30B14C
:1009B000701CFA2E0646F6D3FFF75CFF04E0022116
:1009C000204601F02EFE0025284670BDC046C046D8
:1009D000F8B5394802F00AFB384801250024934E47
:1009E0002946224648F20003B0470326904F334879
:1009F0002146324648F20003B847304848F2000129
:100A000001F00FFE2C48C01C02F0F0FA0C482946F9
:100A100022462B46854FB8470948214632462B4689
:100A2000834FB84702270648294622463B467F4D5A
:100A3000A8470348214632463B467D4CA047F8BDB7
:100A400000140048F8B5774802F0D0FA764C00253B
:100A500001261023754F204629463246B8472023E9
:100A6000204629463246B84740232046294632468A
:100A7000B8478023204629463246B847F8BDC046CD
:100A8000B0B50D4802F0B2FA0C4C01210025204609
:100A90002A4642F2000301F0CFFD032220462946F8
:100AA00042F2000301F0E7FD204642F20001B0BC33
:100AB00004BC964601F0B5BD1305000000080048CF
:100AC00070470000F0B585B0564802F08FFA564CDA
:100AD000012103910227554D20463A46049740F2E2
:100AE0000013A84700210291032520462A460195BC
:100AF00040F200134E4EB047204640F200114D4ADE
:100B000090472046039E31463A4640F20023F14F7B
:100B1000B8472046029F39462A4640F20023444DFA
:100B2000A847204640F20021424A904720463146DD
:100B3000049E324640F20043E64DA847204639461F
:100B4000019A40F200433A4DA847204640F2004146
:100B5000384A904720460399324640F60003DD4D5F
:100B6000A84720463946019D2A4640F60003304EEC
:100B7000B047204640F600012E4A90472046039E8B
:100B80003146049A41F20003D24FB84720460299F9
:100B90002A4641F20003FB4FB847204641F20001CC
:100BA000F94A904720463146049E324642F20003FD
:100BB000F34FB847204602992A4642F20003F14F0C
:100BC000B847204642F20001EF4A90472046039F73
:100BD0003946324644F20003E94EB0472046029EB1
:100BE00031462A4644F20003E64DA847204644F227
:100BF0000001E54A904720463946049A48F200032E
:100C0000DF4DA84720463146019A48F20003DD4DEA
:100C1000A847204648F20001DB4A05B0F0BC08BCFA
:100C20009E461047120500000004004839260008BF
:100C300077260008232600080C48006840F2E831B7
:100C4000B0FBF1F0401E010E00D0FEE70849094A52
:100C50005060094803680B40032189075918016057
:100C600000209060072010607047C04604000020FC
:100C7000FFFFFF0010E000E020ED00E0F0B587B0DE
:100C800037480021017041600E460191354940F21C
:100C900010608847344D35492846884703AC3449AD
:100CA00020468847472002902080324805900496CD
:100CB000314A2846214690470127304A284639467E
:100CC00000979047142002212D4A90472D4928462D
:100CD000884740F21060401C224988472A4E30461F
:100CE0002249884703AD2846214988470298288031
:100CF00020480590019C0494304629461E4A90479E
:100D0000304639461D4A90471520032529461C4A7E
:100D1000904730461B49884740F21060801C1149BB
:100D200088471A4E30461149884703AF3846104964
:100D3000884717483880174805900494304639464C
:100D40000D4A9047304600990C4A90471620294694
:100D50000B4A904730460B49884707B0F0BDC04664
:100D6000F0000020ED2F000800400140893000080D
:100D7000D5310008E7030000FD300008B13100085C
:100D80002D2D0008F33000080044014000480140C8
:100D90001F1C00000F270000FEB502901C20022738
:100DA0003946009701F0C2FF744802F01FF909208C
:100DB000C50601240426019628462146324601F044
:100DC00005FC284639462246334601F035FC00270B
:100DD000284639462246334601F04DFC082628466F
:100DE0002146324601F0F2FB28460099224633465E
:100DF00001F022FC284639462246334601F03BFCEE
:100E0000144802F0F3F8144C204602F039FA204658
:100E1000029902F003FA2046394602F0ABFA204666
:100E2000394602F0BCFA2046394602F08EFA2046D6
:100E3000019902F097FA2046314602F0A8FA2046BE
:100E400002F038FA0521204603B0F0BC04BC9646F7
:100E500002F04EBA1107000000440040F8B51B4CE8
:100E6000204602F0C3F8204602F0C0F8184F0124D3
:100E70004025434E3846214622462B46B0470026A1
:100E800003220092384631462B4601F0F4FB3846E7
:100E9000294601F0C6FB02228025384621462B4612
:100EA000374FB8470A4F38463146009A2B4601F073
:100EB000E2FB3846294601F0B6FB88483146224617
:100EC00044F200032E4CA047F8BDC04616050000B2
:100ED0000014004839260008FEB5284802F086F8BC
:100EE0000920C40601260025254F204631460296DA
:100EF0002A4640F60003B8470322019220462946BD
:100F000040F600031F4FB847204640F600011E4A36
:100F10009047204631462A4641F20003184EB0471A
:100F200020462946019F3A4641F20003154EB0473C
:100F3000204641F20001144A9047204602992A4671
:100F400048F200030E4EB047204629463A4648F282
:100F500000030C4DA847204648F200010A4A90477A
:100F6000204640F60001084A9047204641F2000121
:100F7000054A03B0F0BC08BC9E46104711050000AE
:100F80003926000877260008232600080248002199
:100F90004170FFF765BBC0463C010020F0B58FB043
:100FA00007A82021FFF77BF90024022520462946C7
:100FB00000F0AAFD0028F9D000200221059000F0E1
:100FC00099FD46203E493F4B562805D00A18463A1F
:100FD00012881A52801CF7E701223A494A70D14B15
:100FE0003948C01C04900A200390A6480446C8341F
:100FF0000294283001900692104600285DD00879AE
:1010000040B10020087101204821082200F068F951
:10101000C44B2C49187800284DD0059919700498B4
:10102000082914D08B0007AC0022E250E3181825E1
:101030001446042A07D0F8272F40865CBE40341996
:10104000F835521CF5E71C60001D491CE8E70898BC
:10105000039BB0FBF3F00999B1FBF3F1194A9061DE
:10106000D1610798B0FBF3F0864988600199029A34
:10107000059B062B18D00860069C9C401568A8426A
:1010800002D8156CA84208D2104EB57825433446D4
:10109000A5701031121D5B1CEBE70C4DAD782C4296
:1010A000F7D0A543094CF3E70649069888710598DF
:1010B00048709C4BA1E748789FE70FB0F0BDC04651
:1010C0003E010020240200207301002000000020C7
:1010D000024842F2000101F0A8BAC04600080048E8
:1010E00070477047F0B589B00024654D2046294609
:1010F00040F20012FFF736FA287808B1072802D329
:101100005F4906200870697840F2C8125D4B99501B
:10111000E97840F2D01299505B4908700695062C88
:1011200000D19FE0611D685C08B1642801D30020F4
:10113000685422461532A95C09B1642901D3002103
:10114000A954A2004F4FD31940F2D812985000264C
:1011500040F248129E5040F218201950C8201E50EC
:1011600040F208115E5040F288155E510294200151
:10117000C41966635819019098180790581804907C
:1011800034340594C83303930320C44318213246F2
:10119000354624B3069B08951D198D23EB5C8B40C7
:1011A00030461746079A16689B1913603A46DD23A6
:1011B000EB5C8B40059F3E689B1906463B60BD2358
:1011C000EB5C8B401E185D23EB5C8B409A182D2343
:1011D000EB5C089D8B405D190839641CD9E70498C5
:1011E000026003980560019F3E60284B9D4202D338
:1011F00028498D4204D91146264A026015460A46FE
:1012000029469A42029C1E4D05D33046214EB242D9
:101210000646039802D9049A13601A46914203D2F3
:101220001346049A116003600798006840F2F411B5
:10123000884202D3164A904202D91548079A106094
:101240008E4202D3124A964202D9396040F2F41615
:10125000B04202D23860079806600698001D0690DA
:10126000641C5CE725200649085C40F25822054BC7
:1012700098502720085C40F25C21585009B0F0BD1E
:10128000B40500209402002001000020E02E0000A0
:10129000905F0100D0DD060070B56E4C10210E4E3F
:1012A0002046B0470D4D287020212046B047687079
:1012B00040212046B047A87080212046B047C0009A
:1012C000A9788900014368784000084329780143E0
:1012D0000F20884370BDC0465B1400083801002011
:1012E000B0B5104B00251D700F4B1D700F4C627177
:1012F0002571E17003236370207090000C4A107018
:10130000090AA170401D0B4908700620FFF786F9F5
:10131000A071000AE07108212046B0BC04BC9646CA
:1013200000F002B97201002070010020B50A00200F
:10133000B40A002071010020B0B5464C07283DD802
:10134000820001A39A18974600F00EB800F012B878
:1013500000F016B800F01AB800F01EB800F022B87D
:1013600000F051B800F024B82046012955D140F2D0
:1013700000114DE02046012952D140F2002147E002
:10138000204601294FD140F2004141E02046012989
:101390004CD140F600013BE02046012949D141F201
:1013A000000135E02046012946D142F200012FE03C
:1013B0002046012943D148F2000129E0394D204659
:1013C00040F20011A847204640F20021A8472046DD
:1013D00040F20041A847204640F60001A8472046B9
:1013E00041F20001A847204642F20001A8472046EA
:1013F00044F20001A847204648F200012A46B0BC4A
:1014000008BC9E461047204601291BD144F200012A
:10141000B0BC04BC964601F006B940F2001113E0DE
:1014200040F2002110E040F200410DE040F60001E2
:101430000AE041F2000107E042F2000104E048F254
:10144000000101E044F20001B0BC04BC964601F08A
:10145000E8B8C04600040048704780B501F0E7F8DE
:10146000411E884180BD000070B52D4C02250D4EF7
:1014700020462946B04700F03BF801212046B047FE
:101480002846FFF78BF92046294601F0CCF828467C
:10149000FFF784F920462946324670BC08BC9E46B8
:1014A0001047C04623260008B0B51D4C0225204633
:1014B000294601F0B6F800F01BF80121204601F0A2
:1014C000B2F82846FFF76AF92046294601F0ABF842
:1014D0002846FFF763F920462946B0BC04BC96466F
:1014E00001F09FB8EE48002101230A4601F0A4B89C
:1014F00070B5EB4C00250126204631462A4633467E
:1015000001F09AF8032220462946334601F0B3F849
:10151000044848F2000170BC04BC964601F081B852
:101520000014004800080048F8B50C46009000255B
:10153000C54E084FA5420CD00098415D304601F0E1
:1015400099FE3046394601F0C2FE0028F9D06D1CE4
:10155000F0E7F8BD060700000348016811B1016813
:10156000491E01607047C046F80A002030B4334875
:10157000026801210A43026002689207FCD54268B2
:101580002F4B1340436042682E4B13404360026868
:101590002D4B13400360C26A0F239A43C262026B51
:1015A00040F203139A4302630A04036B93430363F9
:1015B000CA07036B93430363426B8A43426300226F
:1015C000826002680A430260204B022204685D1EAA
:1015D0009D4202D214402B46F8D003689B0700D4EA
:1015E000FEE71B4B1C680725AC431C601C681443BA
:1015F0001C604368436043684360436843604368DA
:10160000144C1C4044604368134C1C4344600B065C
:1016100004681C43046003689B01FCD543680324F1
:10162000A343436043681343436042681207FCD5F9
:10163000C806002130BC01F0ADBBC046001002401E
:101640000C00FF08FFFFC277FFFFF2FEFF0400005F
:1016500000200240FFFFC2F70000040810B50A4C4A
:101660000121204601F0ACFD68B10121204601F0C6
:10167000A3FD0021204601F005FD0448006810BCD0
:1016800002BC8E46004710BD00200040140200201E
:10169000F8B5164D01242846214601F091FD012898
:1016A00003D10121284601F087FD31492031002274
:1016B0000F4B1646062E13D0985D0F46183F28B1E3
:1016C00038680D68A84203D2401C05E03A6004E087
:1016D00008488455002098553860091D761CE9E7B4
:1016E0002349486808B1401E4860F8BD00400140E9
:1016F000440200205602002010B5074C012120466C
:1017000001F05EFD012806D10121204610BC04BC79
:10171000964601F051BD10BD00440140B0B5134DD7
:1017200001242846214601F04BFD012803D1012167
:10173000284601F041FD0E4884700178042901D843
:10174000491C02E00B490C70002101700A490A781B
:1017500022B14278092A04D8511C00E000214170CE
:10176000B0BD00220A704270B0BDC04600480140C2
:10177000F00000202802002025020020B0B51D4CFA
:10178000324D2046294601F0D1FD30B11A4800689B
:1017900080472046294601F0B5FD184D20462946D0
:1017A00001F095FD012806D12046294601F087FD6C
:1017B000114800688047124D2046294601F0B6FDC9
:1017C00030B11048006880472046294601F09AFD54
:1017D0000D4D2046294601F0A9FD48B10948006891
:1017E000804720462946B0BC04BC964601F08ABD1D
:1017F000B0BDC046003801400C02002003070000C5
:10180000070007071002002006000607B0B50E4CBF
:101810000E4D2046294601F089FDA0B120462946FB
:1018200001F070FD204601F021FD09490A78531CA2
:101830000B708A18D0704878DAB2824203D3012044
:10184000887000200870B0BD004400400500050706
:1018500070010020B0B50020064CA047064D28605E
:101860000120A04768600220A047A8600320A0478D
:10187000E860B0BDC52E000828010020B0B5084CB6
:1018800080252046294600F0CEFE2046294600F05D
:10189000C8FE20462946B0BC04BC964600F0C3BE34
:1018A000001400486748016808220A430260016882
:1018B0000907FCD4016804220A4302600168490751
:1018C000FCD4704702280ED0012818D10F20000543
:1018D0000B4A136883431360090509180140106817
:1018E00008431060704703200005054AD36883430E
:1018F000D360090509180140D0680843D0607047DB
:101900002C240140411E8841C0024E490A6840F61D
:1019100000039A43101808607047C04610B5054C84
:10192000204601F077FB204610BC02BC8E4601F039
:1019300067BBC046090300004248016840F200123C
:101940000A4302607047C0463E480168C90703D198
:10195000016801220A4302607047C046012803D093
:10196000022809D1064800E00448364A13680340BB
:1019700013601068084310607047C046FFFFF1FF16
:10198000FF8FFFFFB0B5214B05280AD8052444433B
:101990000846A0401F25A5409C6AAC4304439C62B6
:1019A0001AE00B280BD8052444431E3C0846A040EF
:1019B0001F25A5405C6AAC4304435C620CE0102820
:1019C0000AD2052444433C3C0846A0401F25A540BC
:1019D0001C6AAC4304431C62092909D8032048430C
:1019E0008240072181405868884310435860B0BD49
:1019F000122909D8032048431E388240072181401C
:101A00001868884310431860B0BDC0460C240140DC
:101A100003210906234A13688B43136011680143AD
:101A200011607047C107074904D0012292050B6875
:101A300013430B60800704D5012040050A68024368
:101A40000A6070470824014040F200120346134028
:101A500091B1144913B10B6813430B60420504D5CF
:101A600040F200420B6813430B60800718D54868AA
:101A7000022202434A6070470A4923B10A6840F2D1
:101A800000139A430A60420504D50A6840F20043F5
:101A90009A430A60800703D5486802229043486051
:101AA0007047C04604240140142141433C480A5871
:101AB000012313430B5070471421414338480A58FF
:101AC000202313430B50704710B5142242430D4995
:101AD000521853680124A34353600023536093605A
:101AE000D360136180000F228240086810430860B1
:101AF00010BDC04680008140024802680A4302606F
:101B00007047C046040002408000814002480068DF
:101B10000840411E8841704700000240B0B51422C1
:101B200042431F4813580124A343135013180C6851
:101B30009C608C68DC600C8A5C60135843F600740F
:101B4000A3434C681C43CB6823434C691C4314508B
:101B50000B7E5B1E5C425C41A30114584025AC43E4
:101B6000E31813504B7E5B1E5C425C41E30114584A
:101B70008025AC43E3181350897E4B1E994109011F
:101B800013581024A34359181150B0BD14214143D8
:101B900003480A5844F200039A430A507047C0466B
:101BA0000800024010B5144608463F490A220A7050
:101BB0000722214601F09EFD012804D1044801F0CE
:101BC00013FE012801D0032010BD002010BDC04627
:101BD000204E0000F8B506460F4CA088000A16D12A
:101BE000A0880527032810D30D460092A188264817
:101BF00001F0FAF848B9244908783070481C286088
:101C0000A088801E0099088000273846F8BD03A0F0
:101C10000C499C22FFF746FEB40100207573526305
:101C200076427566666572506F73203C204D425F48
:101C30005345525F5044555F53495A455F4D415893
:101C400000000000843D0008B0B5174D6B780BB163
:101C5000052516E00124EC804B1EAB601870E88867
:101C60008018E880E988184601F0BEF8E9884A1C27
:101C7000EA80054A5054AC7000252846214601F000
:101C80009BFB2846B0BDC046FC0A002010B50120D1
:101C90000024214601F090FB03484470204610BC0C
:101CA00002BC8E4601F014BDB401002080B50020B6
:101CB000014601F081FB80BC01BC864601F0B0BB4F
:101CC00010B5064C2078012805D10548806880476A
:101CD0000020207010BD062010BDC0460800002066
:101CE000F4010020F8B50C460988032505292FD1F9
:101CF0000279C17809028E18711E89B2314B99425E
:101D000026D8811C00918778417800252580012301
:101D1000037023885B1C23805307B2B2D60803B13B
:101D2000761C009B46702088401C20800802C01949
:101D3000401C81B218462B4600F0E8FA20B1F8BCEE
:101D400002BC8E4601F030B8F0B22188081820801D
:101D50002846F8BDF8B50C460988032505292ED17B
:101D60000279C17809028E18711E89B2154B994209
:101D700025D8811C00918778417800252580022391
:101D8000037023885B1C23805307B2B2D60803B1CB
:101D9000761C009B46702088401C20800802C019D9
:101DA000401C81B2184600F001FB20B1F8BC02BC17
:101DB0008E4600F0F9BFF0B221880818208028462E
:101DC000F8BDC046CE070000F8B50C4609880325CB
:101DD000052923D10279511E7C291FD8831C8178C3
:101DE000477800252580032606702688761C2680E5
:101DF000560046702088401C208038024018401C45
:101E000081B218462B4600F0F7FA20B1F8BC02BCAC
:101E10008E4600F0C9BF2088801920802846F8BD72
:101E2000F8B50C4609880325052928D10179C2781F
:101E3000120251184A1E92B27B2A20D8821C0092AC
:101E40008778437800252580042202702288521C5E
:101E500022808AB2560046702088401C20801802DA
:101E6000C019401C81B2009800F096FB20B1F8BC6C
:101E700002BC8E4600F098BF20888019208028463A
:101E8000F8BDF8B5054608880A2841D30C462879DC
:101E9000E97809020F18781E80B203267C2838D80A
:101EA000287AE97909020818411E89B2782930D8C0
:101EB000697A82B2500081422BD1A87969790902EE
:101EC0000818411CA87800906E7828460A3089B21C
:101ED000012300F091FAB0B9BAB23002009940186B
:101EE000411CA81C0026268017232B7023885B1C0E
:101EF000238057006F7023885B1C238089B2334690
:101F000000F07AFA38B1F8BC02BC8E4600F04CBF43
:101F100000263046F8BD2088C0192080F9E700006F
:101F2000B0B50C4605490D88401C891C2A46FEF7B1
:101F300057F9681C20800020B0BDC046C4010020B5
:101F40001CB50988032405291AD10179C1B9827801
:101F50004378C178FF2900D091B918028018421C3B
:101F600001A800244470FF394B424B41037091B2E9
:101F70000122134600F0CAF910B100F015FF044623
:101F800020461CBD80B50988052910D1817842788A
:101F900012025118491C89B2C01C0122134600F0DC
:101FA0002BFA30B180BC02BC8E4600F0FDBE03208F
:101FB00080BD002080BD70B50C460A880321062A2A
:101FC00024D30679C27812029519AAB2D3087607EB
:101FD00000D05B1C6D1EADB22D097A2D16D8457947
:101FE000DBB29D4212D1817843781B025918491CFB
:101FF00089B2801D012300F089F920B170BC02BCB8
:102000008E4600F0D1BE052020800021084670BD1C
:10201000B0B50C460A880321062A20D302794379F9
:1020200055062D0EAB421AD1C3781B029A18531EC7
:102030009BB2772B13D8817843781B025918491C1F
:1020400089B2801D92B2012300F0D6F920B1B0BC54
:1020500002BC8E4600F0A8BE052020800021084664
:10206000B0BD0000F8B50546022091B3CC081E2C87
:102070002FD8069C524E3170012D15D04DBB254DE9
:102080002548264FB760F0603561214870611F48D0
:10209000B0611D48F0611B483062084611461A467F
:1020A000234600F091F813E0134D1448144FB76025
:1020B000F06035610F4870610D48B0610B48F06108
:1020C00009483062084611461A462346FFF76AFD62
:1020D00000B1F8BD01F0F6FA20B1384801210170D5
:1020E0000020F8BD0320F8BD8D350008C535000877
:1020F00081340008D51B0008491C0008AD1C0008ED
:102100008D1C0008D13800081D390008413800082E
:102110000522000879220008F9220008DD220008C3
:102120007CB52648007808B1062445E001A801F0F6
:10213000BDFA002401283FD101A80078022812D05E
:10214000012839D11E4D6B69681C294624312A1D8E
:10215000984788BB68782978884200D060BB022005
:1021600001F0B6FA28E0164D6A6A1178A9700023CA
:102170000120144C802B0AD0E65C46B18E4201D07F
:102180000833F7E7E0184368291D10469847697837
:10219000002489B158B10121A980A97880220A437D
:1021A000696A0A70A9884A1CAA806A6A5054AA8877
:1021B000696A28782B69984720467CBD0800002072
:1021C000F40100200C00002010B514460846082237
:1021D000214601F08FFA01280ED144F600308442E6
:1021E00001D9232003E060000549B1FBF0F080B283
:1021F00001F0FAFA012801D0032010BD002010BD23
:10220000A07F1700F8B506460F4C6088000A16D16B
:1022100060880527042810D30D46009261882E4857
:1022200000F0E2FF48B92C4908783070481C28605B
:102230006088C01E0099088000273846F8BD03A0BA
:102240000C499C22FFF72EFBE801002075735263B6
:1022500076427566666572506F73203C204D425F12
:102260005345525F5044555F53495A455F4D41585D
:1022700000000000053E0008B0B51E4D2B78012B74
:1022800026D10124AC804B1EAB601870A888801842
:10229000A880A988184600F0A7FFA9884A1CAA8030
:1022A0000D4A5054A9884B1CAB80000A5054A868B2
:1022B000007801F08FFAA888401EA880A868401C0A
:1022C000A8606C7000252846214601F075F800E0F2
:1022D00005252846B0BDC046FC0A002080B505484B
:1022E00000210170012001F067F880BC01BC864626
:1022F00001F0AEB8E801002080B50020014601F0F1
:102300005BF880BC01BC864601F08AB8FEB5144675
:102310000246491E88B20019042824D8601E0825E8
:10232000019590FBF5F0451C0020F3B1012B1BD16A
:1023300000901D4B280435D06D1E02921078224665
:10234000019F541E12040BD03A0609D0012202400C
:102350008EB29A55491C7F1EC0B240082246F0E753
:10236000029A521CE6E70120FEBD00900820019071
:102370000D4F280416D002926D1E002622460198A9
:10238000541E12040AD0020608D08AB2BA5CB240C7
:102390001343761C491C401E2246F1E7029A137033
:1023A000521CE6E70098FEBDFC0B0020F0B5491E6C
:1023B0008BB2DC0801217D2C1BD39B1840F2EC343E
:1023C000A34216D8511E082391FBF3F14C1C0021A7
:1023D00025040ED0641E16461D46721E360404D017
:1023E0006F1E2D0616463D46F7D100250570401C90
:1023F000EEE70846F0BD0000FEB515460646481E4D
:1024000087B201205C4A974200D89DE07A195B4C64
:10241000A24200D998E041F27072BA1A584C626038
:10242000012B0CD023BB5448401C874254D1022DB1
:1024300052D1500055490968524A11525CE001924C
:10244000009065700522D24340F2D07353434D484B
:10245000C3187C001B192C4622040BD032781202C0
:102460001A80707810181880B61C9B1C641EF3E745
:102470000020FEBD4048401C87423FD101984000EB
:10248000404909182806C20D404C2046FDF7A8FE19
:10249000206808B1072801D30620206002AE307002
:1024A00000250127284631463A46FEF787F830785E
:1024B000374908700821081AFF21C14035480170CA
:1024C000384631463A46FEF74DF8206840F2007132
:1024D000401820602846FEBD41F2A370081A303033
:1024E00080B2952831D85000264908189100274A13
:1024F00051186A00FDF774FE002227E041F2A37034
:10250000081A80B2652800981ED8019840001D491D
:1025100009181B48047866011B488719384608309B
:102520002A06D20DFDF75CFE01201749885101985B
:102530007860601CC1B200221F291346114600D8E2
:1025400001460F4801701846FEBD01220520C04318
:1025500040F2D07141430B484018790040182904DB
:1025600007D04178317001787170B61C801C6D1EE7
:10257000F5E71046FEBDC0466F170000581B00006F
:102580001C020020000C0020B40600209402002051
:10259000010000200000002010B50346481E81B253
:1025A0000120084CA1420BD38918074CA14207D83F
:1025B0000020110404D0587018709B1C521EF8E7BC
:1025C00010BDC046B80B0000BC0B0000FCB501916B
:1025D000016A0090446A00252E46202D0CD0174633
:1025E000F740FF0705D0019FAF400F23AB40994351
:1025F00039432D1D761CF0E708250026202E0CD02F
:102600001346EB40DB0705D0019BB3400F27B740D3
:10261000BC431C43361D6D1CF0E700980162446208
:10262000FCBD8162704781617047C162704700697B
:102630000840411E88417047FEB50293019202682E
:102640000090C56800263746202E10D0029BFB4024
:10265000DB0709D0019BB3400324B440A5431D43CD
:102660000B46B340A2431A43B61C7F1CECE700980C
:102670000260C560FEBDF8B5012902D14168194369
:1026800001E0416899434160009081680024032083
:102690002646202C0CD01F46F740FF0705D01746D2
:1026A000A7400546A540A9433943A41C761CF0E782
:1026B00000988160F8BD000094B00CA8202106911C
:1026C000FDF7EDFDD44C0020E0812072E071D3498C
:1026D000FF250D70582132220892024670290AD037
:1026E000CD4B9B18089C1855069C1855CA4C605039
:1026F000091D521CF2E7FEF739FFFFF7ABF8FEF7B2
:10270000DFF9FEF799FAFEF7BBF9FEF79BF9FEF742
:10271000D9F9FEF7A3FBFEF7DFFBFEF7AFFA41F2B4
:10272000C020FEF739FBFEF751F9FEF7DBFCFEF7A0
:102730002DFC00266661FEF7AFFD01460096E12004
:102740004302304603963246FFF78CFCFFF7B8FA97
:10275000B24A507838210791605440F20071411814
:102760002182AF4B19600821081AC540157040F24C
:10277000D81018181121C94309910C3151B1A64A3A
:10278000521803683F241355036C45241355001D4C
:10279000491CF3E7A3484021FFF743FFFEF7FEFB88
:1027A00040F2C81003999E4D295001209A4C0A907E
:1027B000A07061729C4A50785170984E31780840F0
:1027C000A072B0780840B070C0B2FDF7ECFFB078EE
:1027D000607358343435767836B12868FDF758FE82
:1027E00001C41035761EF7E740F248108C490818EE
:1027F00002908E48C01C01908D4844F20001FFF702
:1028000016FF854B002800D0B3E099789C7A864863
:1028100042780B94A24217D1D87808435FD003982E
:1028200058800798185C19463231824A002856D0E1
:102830000023099C0B550B700C192373A37108C25C
:10284000754B401E491CF1E71846079BC35CC478D2
:10285000059404910C430FD06F4C32341E46754FD3
:1028600056B10020099D6055207065192873A87124
:1028700001C7761E641CF3E700246E4EA3422BD0E2
:102880000B98E0400A9908401546E5400D40854206
:1028900009D9614807192C2039540598B8B1069810
:1028A00039543F200CE014D25B48071926200A99BE
:1028B00039540846049949B10146069839543920DB
:1028C000385C40F2E8314843306002E00146089845
:1028D0003954361D641CD1E700204F4B588000242A
:1028E000544A0798185C844241D21F190898385CF2
:1028F000A8B338463230002506997D54156005701E
:102900000A9EA6402620385C0B9260B12637E0B2C2
:102910000121FEF711FD424A40F2C813D158F0B22E
:102920000843D0500DE02C20385CD8B12C37E0B2F1
:102930002946FEF701FDF54940F2C812885CB04314
:1029400088503D70F04909780140F1484170C9B2A2
:102950000120FDF743FEFEF791FFEA4B0B9A121D93
:10296000641CBEE7E94840F2C8114058EAE70A98FB
:102970001870E74840789872FFF7D2FBE149087970
:1029800040B103980871887920B1012048210822BC
:10299000FEF7A6FCDF48007800286CD00399DD48DC
:1029A00001700198082914D08B000CAC0022E25071
:1029B000E31818241546042A07D0F8262640875C19
:1029C000B7407D19F834521CF5E71D60001D491C05
:1029D000E8E764210C980B91B0FBF1F20A20424326
:1029E000CA4CA2602346C83328340025062D23D0C4
:1029F00022600A9FAF40C4498E7819688A4201D983
:102A00003E4302E0374202D0BE43BF498E701034CD
:102A10001B1D6D1CEAE7C0462402002000000020B8
:102A20009402002000140048B40500207301002027
:102A300000080048100100200F990B9DB1FBF5F133
:102A40004143B24A51610D99B1FBF5F14143AD4AA1
:102A500094690B1B0022A14200D21346AB49CB6004
:102A60000E99B1FBF5F14843A649C969401A00D255
:102A70001046A6490861FDF71DFF002840D0FEF76B
:102A800027FBFDF7E9FD00F0D1FAA04C3434002516
:102A90002E469D484078864232D20998800000191F
:102AA000406CFDF7F5FC9C49FDF7FEFB9B49FDF7EB
:102AB000FBFB014693484719B86D00F06FFFB865FE
:102AC000FDF7A2FC2060411C02D100202060B86507
:102AD0008F494919DC228854020ADB23CA54020CAC
:102AE000DA23CA54000ED9228854D9312846D93065
:102AF00080B20422FDF762FD10342D1D761CC8E75C
:102B000087490878F0B300240C70804D3035854E2D
:102B100002980B907B4B7C48407884422CD20998D9
:102B2000800047193088FDF721FE764B78641978CC
:102B300081B10A99A140DA7A0B9B1B68984204D9AB
:102B40000A437049CA720B4604E011426D4B01D032
:102B50008A43DA720A21B0FBF1F03A6CB2FBF1F26F
:102B60004243B2FBF1F02860002001C610350B98FB
:102B7000001D0B90641CCEE763488178D87A084327
:102B8000187301E05F4B187B0106674C08D0597B36
:102B9000C0B2884204D0FDF706FE5A4B187B58732A
:102BA000187A41016258002A62D0611848684128A9
:102BB00012D889688000554A11500A0E544D4319A5
:102BC0009F382A541A469C3A11701A469D3A0C0AAC
:102BD0001470554C9E3B3DE0512812D88968800006
:102BE0004A4A11500A0E4A4D4319AF382A541A4620
:102BF000AC3A11701A46AD3A0C0A14704A4CAE3B0E
:102C000028E0612812D889688000404A11500A0ED5
:102C10003F4D4319BF382A541A46BC3A11701A4620
:102C2000BD3A0C0A1470404CBE3B13E0712826D804
:102C300089688000354A11500A0E354D4319CF3846
:102C40002A541A46CC3A11701A46CD3A0C0A14701E
:102C5000354CCE3B090C1970291880B20422FDF7BF
:102C6000ADFC284B187A4101002262500A99597133
:102C7000401CC1B21F2900D900201872BCE597285A
:102C80000BD074280DD0962812D0722816D1087A4D
:102C90001D49097801409972E4E70A98D87000202C
:102CA0000AE0087A1849097801401948C170D9E743
:102CB0000A989870144800789872D3E785280DD840
:102CC0008A680346713B1249CA54D1B284000F4D41
:102CD00029510C4C0019144C3D380EE09528C1D8F0
:102CE0008A680346713B0A49CA54D1B28400074D31
:102CF0002951044C00190C4C4738027098B2FDF76A
:102D00006DFCAEE7240200200000002094020020A9
:102D1000B40500207201002000007A4400006145E3
:102D20003C01002050010020B406002070B540B2E4
:102D3000002817D4032302469A43144BD45885071E
:102D4000ED0EFF26AE40B4438901C9B2A94021432C
:102D5000D1501F21014001228A40400980000C49C6
:102D6000425070BD8207D20EFF2494400F230340CF
:102D7000083B0320834304481D58A5438901C9B279
:102D800091402943195070BD1CED00E000E400E0C3
:102D900000E100E0024A0A40024302480260704734
:102DA00080FFFF1F08ED00E040B1072803D0012895
:102DB00003D10220704706207047042070470000AE
:102DC0000A2801D2302102E0102803D23721081846
:102DD000C0B2704702A0034940F2D012FEF762FD74
:102DE00030000000843D000800220B0405D0037869
:102DF000D218D2B2401C491EF7E75042C0B2704709
:102E000070490A684CF200039A430A60CA6A2C4B64
:102E10001340CB62092851D8820001A39A18974623
:102E200000F012B800F015B800F01DB800F01EB8A0
:102E300000F01FB800F021B800F023B800F025B86A
:102E400000F032B800F025B801200004CA6A8243BD
:102E500003E001200004CA6A0243CA62C86A40F261
:102E60000012904329E00868086022E008680860C2
:102E700014E0086844F2000219E0086844F2000215
:102E80000AE0086848F2000211E0086848F200020F
:102E900002E008684CF2000202430A600120C00709
:102EA000CA6A0243CA6204E008684CF200020243A4
:102EB0000A60CA6A40F200101043C8627047C046F8
:102EC000FFFEFE7FF8B501463E4B18680C2202401B
:102ED0003D48082A044618D11A689202120F0F2A98
:102EE00001D0941C00E010241D682D0101D5113281
:102EF00014461A68D20301D4344A05E09A6A0F25B1
:102F000015406A1CB0FBF2F254431D6818681A6839
:102F100005291FD800902D062D0F2DA77F5D254672
:102F2000FD409204520F2E4FBE5C2A46F2408E00A6
:102F300001A080198746C04600F00AB800F011B819
:102F400000F00AB800F00EB800F00EB800F014B8A7
:102F5000224607E0002205E000984005400F385C5B
:102F6000C5402A461046F8BDD86AC0051AD4D86AAA
:102F7000C00320D51C48F8BDD86A8007F2D0D86AB3
:102F80000321084001282246ECD0D86A084048F2C4
:102F900000020228E6D0D86A084003280A4800D078
:102FA0000020F8BD18680004800FD96A002904D4F5
:102FB000B2FBF0F2D6E70B48F8BD401CB5FBF0F2CF
:102FC000D0E7C0460410024000127A0000093D001C
:102FD00000000000000000000102030406070809C9
:102FE000383D0008809FD500003FAB011F21014004
:102FF00001228A4080090C494358134343507047CB
:103000001F21014001228A40800907494358934308
:10301000435070471F21014001228A408009024924
:1030200043581343435070470010024070B5134893
:10303000417803290BD8024614320023102B17D0F5
:10304000C418648815682C1910C29B1CF6E700216F
:103050004170024614320A4B0C46102C0BD01D5BFB
:103060001668B608751B00D20D4620C2A41CF4E7F2
:10307000491C417070BD0121017070BD3C010020F0
:103080006A0200204162704710B5154C44498842DD
:1030900013D01449884212D0EC49884211D03D49DE
:1030A000884213D03D4988420DD03E4988420CD019
:1030B0003949884213D1F63408E0E41D06E0F934BA
:1030C00004E0FD3402E0641D00E0A41D2046FFF78B
:1030D000A1FF204610BC02BC8E46FFF791BF10BD79
:1030E0000B030000001000400168012291430160C1
:1030F0007047016801220A430260704710B50A88D0
:103100008262244A904202D0234B98420BD103683A
:103110007024A34303604B8804681C4304608B88BD
:1031200004681C4304608B68C36290420FD113682B
:1031300040F20034A3431360CB8814681C4314602E
:10314000097B0163416901220A43426110BD124AB1
:1031500090420BD0C94A904208D0104A904205D004
:103160000F4A904202D00F4A9042EBD1026840F2DF
:1031700000339A430260CA88036813430360074A16
:103180009042DDD0074A9042DAD0054A9042D7D02B
:10319000D8E7C046002C0140000400400040014038
:1031A0000048014000440140C2688A43C260704741
:1031B000C2680A43C260704702698A43026170476D
:1031C000C2680A40531E9A4100690840411E884166
:1031D0001040704703490022027302604260816020
:1031E0007047C046FFFF0000F0B5FF24094A0A4BB4
:1031F00025460E0409D006787540565D5F5D25466C
:103200007D40401C491E3446F3E72002284380B22B
:10321000F0BDC046383C0008383B0008B0B50D464C
:1032200004467E48844204D02048844205D10220CE
:1032300000E00520FFF746FE00E0002021680904B9
:1032400005D469084018B0FBF5F080B209E06908C0
:1032500040004018B0FBF5F0034901400007400F63
:103260004018E060B0BDC046F0FF0000416A03486E
:1032700008407047014A0A4082627047FF0100001F
:1032800010B56649884204D0084988420BD1084CE1
:1032900000E0054C2046FFF7BDFE204610BC02BCF6
:1032A0008E46FFF7ADBE10BD0E0300000044004087
:1032B00011040000016801220A43026070471F22C6
:1032C0000A4001219140026A0A43026270471F22AC
:1032D0000A4089090958D1400120084070471F223F
:1032E0000A400123934089090A589A430A507047BB
:1032F0001F220A400123934089090A581A430A50A1
:1033000070470000084A914206D1D021425848F245
:1033100000039A4342507047C902C90E01228A40F5
:10332000016A11430162704709340F341F220A40B9
:103330000B049B0D1B58D3408A0D1258C802C00EB7
:10334000C2401A40012010407047026801239A438E
:103350000260026840F200639A43026002680A4316
:1033600002607047026804239A43026002680A43BD
:1033700002607047026801239A430260426843F288
:1033800000039A43426042680A4342607047026801
:1033900008239A43026002680A4302607047026889
:1033A00001239A430260026841F200039A430260DB
:1033B00002680A430260704770B50E460921CC06C8
:1033C000CB4D0521012808D12846FFF791FF204663
:1033D00040F20011FFF725F907E02846FFF77FFFCD
:1033E000204640F20011FFF71EF906212846012E63
:1033F00009D1FFF77DFF204640F2001170BC04BCEC
:103400009646FFF710B9FFF76AFF204640F2001119
:1034100070BC04BC9646FFF704B9C04600380140B2
:10342000B0B5164C00212046FFF72CFE01252046A2
:103430002946FFF7C1FE20462946FFF7B5FE204684
:10344000B0BC02BC8E46FFF74FBEC0460020004015
:10345000B0B50A4C00212046FFF714FE0125204696
:103460002946FFF7A9FE20462946FFF7A1FE204680
:10347000B0BC02BC8E46FFF73CBEC04600200040F8
:10348000BCB53A4DA87800286AD101A800F028F907
:103490006878002478B1022818D001285ED1FFF79F
:1034A000D7FF01A800780D2828D000243A2828D179
:1034B000EC70AC8052E001A800783A284ED1FFF7BA
:1034C000C7FF0024AC80EC70012018E001A8007850
:1034D0002978884208D1FFF7A3FF002068700120F7
:1034E00000F0F6F8044639E000243A2810D1EC70D8
:1034F000AC8001206870FFF7ABFF2FE002206870FE
:103500002CE001464139C9B2062903D3E14303E067
:103510006C7023E0014637393038C2B20A2A00D332
:103520000846E97801290AD0C1B9A988FF2911D82C
:10353000A9880001E54A50540120E8700EE0A988EE
:10354000E24A535C03435354A888401CA8800024DB
:10355000EC7003E000246C70FFF762FF2046BCBDF6
:1035600003A05149E322FEF79DF9C046B4010020B3
:1035700065536E645374617465203D3D205354411E
:1035800054455F54585F49444C45000080B53E485F
:103590004178491E012902D80021417005E0417897
:1035A000012902D04078022803D1FFF739FF00201B
:1035B00080BD03483C4940F2A712FEF773F9C046AC
:1035C000403D000870B5304E7078002856D1B07874
:1035D000042840D8810001A251188F4600F008B895
:1035E00000F027B800F009B800F02BB800F014B8CC
:1035F00001200021FFF7E0FE2DE0F08830B3F078E5
:1036000001282AD038BBB06800780009FFF7D8FB42
:1036100000F0E0F8012012E00024B470032000F074
:1036200057F8054601202146FFF7C6FEB47028462C
:1036300070BD3A2000F0CEF80220B0700020F0708B
:1036400009E0307800F0C6F8042003E00D2000F017
:10365000C1F80320B070002070BDB06801780F2061
:103660000840FFF7ADFB00F0B5F80020F070B0683F
:10367000401CB060F088401EF080ECE703A00A49CF
:1036800040F24F12FEF70EF9B40100206552637646
:103690005374617465203D3D2053544154455F523D
:1036A000585F49444C450000843D00080B490A78A6
:1036B000012A05D14A780270002008700120704765
:1036C0000020704705480021017001207047C04666
:1036D00002494870012008707047C046C0010020B0
:1036E00010B504463F48FFF7C1FD2070012010BD12
:1036F00000380140FEB502911B2000252946FFF746
:1037000015FB3148FFF772FC0920C606012430463C
:10371000214640F20022FEF759FF02210191304676
:10372000224640F20023294FB847294F3046294608
:10373000224640F20023B8473046214640F200427C
:10374000FEF744FF30460199224640F200431F4FE6
:10375000B84730462946224640F200431C4FB8473E
:10376000304621462A4640F20013184FB84703223C
:103770003046294640F20013154EB0471248FD303E
:10378000FFF734FC174E3046FFF77AFD30460299BA
:10379000FFF744FD30462946FFF7ECFD3046294649
:1037A000FFF7FDFD30462946FFF7CFFD04213046E7
:1037B000FFF7D8FD08213046FFF7E9FD3046FFF757
:1037C00079FD2046FEBDC0461105000039260008DF
:1037D0007726000880B501460248FFF74BFD01201F
:1037E00080BDC046003801407FB5054640F20870F4
:1037F000FFF7FCFB104C2046FFF746FC6E463046B8
:10380000FFF7E8FC0D483080681E02900020019010
:1038100020463146FFF772FC012520462946FFF776
:10382000C7FC13202946FFF781FA2046FFF761FC09
:10383000284604B070BDC046002000400F0E0000B6
:103840001CB51A4C607858BB01A8FFF749FF2078D7
:10385000032823D8810001A251188F4600F01CB81C
:1038600000F004B800F00CB800F016B8002060803A
:103870006088411C61801549019A0A5402200AE0BF
:103880006088FF2806D86088411C61800F49019A32
:103890000A5401E003202070FFF7DAFD00201CBD70
:1038A00003A03D49F022FDF7FDFFC046E8010020DE
:1038B00065536E645374617465203D3D20535441DB
:1038C00054455F54585F49444C450000FC0A0020B1
:1038D000B0B5294D28780024032808D0022802D04A
:1038E00058B9002000E00120FFF7F2FE0446FFF780
:1038F00097FD012028702046B0BD28780028F6D01A
:1039000028780228F3D028780328F0D002482249EA
:1039100040F26512FDF7C6FFA23D000870B5164ED5
:103920003078012822D17078012805D080B9012093
:103930000021FFF741FD0BE0B08858B1B068007876
:10394000FFF748FFB068401CB060B088401EB080F0
:10395000002070BD0320FFF7BBFE044601200025B8
:103960002946FFF729FD7570204670BD03A00A495E
:1039700040F22B12FDF796FFE801002065526376B6
:103980005374617465203D3D2053544154455F524A
:10399000585F49444C450000053E000870B50125BC
:1039A000ED0704004C4020D4441A01D2001B091931
:1039B000C60D4B00F2B2FF2A29D01B0E2CD00002FC
:1039C0000C0228432C43D31ADC40051910D2280AD4
:1039D00002D3401C6D0611D0761EF6058019FF2A11
:1039E00000DA70BDC00DC00570BD694000F022F85E
:1039F00001200543C541521C761CE8E764089C4041
:103A0000C90161408900E7D10124A043E4E71B0E0E
:103A1000440200D0034870BD002AFCD1C00FC0078B
:103A200070BD00BF0000C07F70B50125ED07040028
:103A30004C4022D4441A02D26C40001B0919C60D16
:103A40004B00F2B2FF2A4BD01B0E50D000020C02EA
:103A5000A8432C43D31ADC40051B05D5AD0019D370
:103A60006D08761E521E37D0F605280A01D280193D
:103A700070BD70416D0603D070BD6940FFF794FFC3
:103A80009C4009026140490001D0401E70BD0124E4
:103A9000A04370BD6D081DD001202B0C01D12D0459
:103AA00010302B0E01D12D0208302B0F01D12D012A
:103AB000001DAB0F01D1AD00801CEB0F01D16D00DB
:103AC000401C361A121A6D00680AF5054019012AC1
:103AD00002DB70BD002070BDC036300AC00770BD6B
:103AE0001B0E440201D1FF2B00D1024870BD002AF9
:103AF000F0D070BD0000C07F818283848586878876
:103B0000898B8C8D8E8F919293959697999A9C9D87
:103B10009FA0A2A3A5A7A8AAACAEB0B2B3B5B7B9EF
:103B2000BCBEC0C2C5C7C9CCCED1D4D7D9DCDFE2B8
:103B3000E6E9ECF0F3F7FAFE00C1814001C08041F4
:103B400001C0804100C1814001C0804100C181406D
:103B500000C1814001C0804101C0804100C181405D
:103B600000C1814001C0804100C1814001C080414D
:103B700001C0804100C1814001C0804100C181403D
:103B800000C1814001C0804100C1814001C080412D
:103B900001C0804100C1814000C1814001C080411D
:103BA00001C0804100C1814001C0804100C181400D
:103BB00000C1814001C0804101C0804100C18140FD
:103BC00000C1814001C0804100C1814001C08041ED
:103BD00001C0804100C1814000C1814001C08041DD
:103BE00001C0804100C1814001C0804100C18140CD
:103BF00000C1814001C0804100C1814001C08041BD
:103C000001C0804100C1814001C0804100C18140AC
:103C100000C1814001C0804101C0804100C181409C
:103C200000C1814001C0804100C1814001C080418C
:103C300001C0804100C1814000C0C101C30302C274
:103C4000C60607C705C5C404CC0C0DCD0FCFCE0EDC
:103C50000ACACB0BC90908C8D81819D91BDBDA1A4C
:103C60001EDEDF1FDD1D1CDC14D4D515D71716D6BC
:103C7000D21213D311D1D010F03031F133F3F2322C
:103C800036F6F737F53534F43CFCFD3DFF3F3EFE9C
:103C9000FA3A3BFB39F9F83828E8E929EB2B2AEA0C
:103CA000EE2E2FEF2DEDEC2CE42425E527E7E6267C
:103CB00022E2E323E12120E0A06061A163A3A262EC
:103CC00066A6A767A56564A46CACAD6DAF6F6EAE5C
:103CD000AA6A6BAB69A9A86878B8B979BB7B7ABACC
:103CE000BE7E7FBF7DBDBC7CB47475B577B7B6763C
:103CF00072B2B373B17170B05090915193535292AC
:103D000096565797559594549C5C5D9D5F9F9E5E1B
:103D10005A9A9B5B99595898884849894B8B8A4A8B
:103D20004E8E8F4F8D4D4C8C4484854587474686FB
:103D3000824243834181804000000000010203046D
:103D40002820655263765374617465203D3D20538D
:103D5000544154455F52585F5243562029207C7C81
:103D6000202820655263765374617465203D3D20A0
:103D700053544154455F52585F574149545F454F32
:103D8000462029002E2E2F4170702F4D6F646275D2
:103D9000732F61736369692F6D6261736369692E43
:103DA00063002820655263765374617465203D3D3D
:103DB0002053544154455F52585F494E495420297D
:103DC000207C7C20282065526376537461746520C2
:103DD0003D3D2053544154455F52585F5243562055
:103DE00029207C7C20282065526376537461746599
:103DF000203D3D2053544154455F52585F45525237
:103E00004F522029002E2E2F4170702F4D6F64626B
:103E100075732F7274752F6D627274752E63000046
:103E2000403E000800000020900000001001000843
:103E3000D03E000890000020401B00002C0100082C
:103E4000FF06FF0000A24A0402000000110000006B
:103E5000211F000804000000211E000803000000CC
:103E6000C91D000810000000112000080600000015
:103E7000851F000817000000831E000801000000D5
:103E8000E51C000805000000411F00080F000000AD
:103E9000B71F000802000000551D000800000000C8
:103EA0000000000000000000000000000000000012
:103EB0000000000000000000000000000000000002
:103EC00000000000000000000000000000000000F2
:04000005080000CD22
:00000001FF
